:1000000047C161C128C35FC15EC15DC15CC15BC145
:10001000B4C359C158C157C100C455C154C16DCDF5
:100020004ECD7ACD84CD8ECD9BCDB8CD76167B17B7
:10003000811886198B1A911B961C9B1DA11EA61F49
:10004000AB20B121B622BB23C124C625CB26D127A4
:10005000D628DC29E12AE62BEC2CFF0B000000005F
:10006000A60EF9154C1DF22B3E498A6601020304C7
:100070000506070200FFFF00FF000000000000006F
:10008000FF0000000078FF000C3F96FFFF0000001B
:1000900000000000FF00000000FF00146E96FF004B
:1000A0000000000000FF000000FF001E78FF0000BD
:1000B000000000FF0000FF001EFF00000000FF0026
:1000C000FF00FF000000FF0000FF00FF0000000035
:1000D0000000000000000000000000000000000020
:1000E0000000000000000000000000000000000010
:1000F0000000000000000000000000000000000000
:1001000000000000000000000000000000000000EF
:1001100000000000000000000000000000000000DF
:1001200000000000000000000000000000000000CF
:1001300000000000000000000000000005070A0E9B
:100140001114181C2024282D32373C41474D535997
:100150005F666D747B828A929AA2AAB3BCC5CED721
:10016000E1EBF5FF000000000000000000000000CF
:10017000000000000000000000000000000000007F
:10018000000000000000000000000000000000006F
:10019000000000000000000000000000000000005F
:1001A0000005070A0D1013171A1E2125282C3034BC
:1001B000383C4045494E52575C60656A6F757A7F9E
:1001C000858B90969CA2A8AEB5BBC2C9CFD6DDE404
:1001D000ECF5FFFFFFFFFFFFFFFFFFFFFFFFFFFF4C
:1001E000FFFFFFFFFFFFFFFFFFFFFFFFFFFFFFFF1F
:1001F000FFFFFFFFFFFFFFFFFF00030303040404F3
:10020000050505060607070808090A0B0C0E10125B
:100210001416191C1F2225292D3135393D42474C12
:1002200051565C62686E747D848B9299A1A9B1B9B4
:10023000C2CBD4DDE7F1FBFFFFFFFFFFFFFFFFFFB6
:10024000FFFFFFFFFFFFFFFFFFFFFFFFFFFFFFFFBE
:10025000FFFFFFFFFFFFFFFFFFFFFFFFFFFFFFFFAE
:10026000FFFFFFFFFFFFFFFFFFFFFFFFFFFFFFFF9E
:10027000FFFFFFFFFFFFFFFFFFFFFFFFFFFFFFFF8E
:10028000FFFFFFFFFFFFFFFFFFFFFFFFFFFFFF007D
:1002900011241FBECFE5D2E0DEBFCDBF10E0A0E647
:1002A000B0E0EAE7FCE102C005900D92AA39B1077F
:1002B000D9F720E0AAE9B0E001C01D92AF3FB20734
:1002C000E1F78AD7D8CC9CCE19BC18BC1BBC0895CA
:1002D00020ED37E0019720F0F9013197F1F7FACFDF
:1002E0000895CF93DF93E091F700F0E0E459FF4FDA
:1002F00084918093E2001092CE001092E800109258
:10030000D8009091FC00992351F09091FB009093BC
:10031000D9001092CF001092E90092E001C091E064
:1003200020E030E0682F70E0C92FD0E026173707B3
:100330000CF036C0A091F700B0E0AA0FBB1FAC577D
:10034000BF4FED91FC91E20FF31FE491A9014C0F17
:100350005D1FDA01A852BF4FEC93A091F700B0E007
:10036000AA0FBB1FAC58BF4FED91FC91E20FF31FDA
:10037000E491DA01A851BF4FEC93A091F700B0E0EF
:10038000AA0FBB1FAC59BF4FED91FC91E20FF31FB9
:10039000E491DA01A253BF4FEC932F5F3F4FC6CFDA
:1003A000890F8093E200DF91CF910895811101C000
:1003B0008BCF815090E0FC01E253FF4F2491FC0170
:1003C000EC59FE4F3491FC01E650FE4F849189BDFB
:1003D00038BD2BBD089581E08093CD0093E09093CC
:1003E000FB008093CB0022E02093E6009093F7007F
:1003F0008093FC001092CC001092FA008093F900D8
:100400001092E3008093F6000895CF93DF931F923C
:10041000CDB7DEB79FEF9BBD90E0698359DF1BBC72
:100420006981862F90E00F90DF91CF9151CF80911D
:10043000CD008093B9001092CD001092FE008BE5A4
:100440008093BB0008958091B9008093CD001092F5
:10045000C6008091CD00882319F01092BB0008954A
:100460008091BA008093BB000895EF92FF920F93A2
:100470001F93CF93DF93C82F8B017B01EE0CFF1CE2
:10048000EE0CFF1CD2E3CC2361F0D9BD18BC1BBC21
:10049000C8011EDF19BC18BC1BBCC70119DFC15045
:1004A000F2CFDF91CF911F910F91FF90EF900895C0
:1004B0000F931F93CF93DF931F92CDB7DEB7182F03
:1004C00002E3112301F18091BB0086131CC08091CF
:1004D000F600882321F08091E300811103C009BD5B
:1004E00018BC1BBC8AEF90E06983F2DE19BC18BC13
:1004F0001BBC87E791E0ECDE8091BB00698186132D
:1005000002C01150DECF0F90DF91CF911F910F915C
:1005100008951F93CF93DF93D62F6AE071DB192FD5
:100520006D2FC6DFC091BB00CD1310C080E293E0F9
:10053000CFDE6C2F812FBCDF8091BB008C1306C0F7
:1005400080ED97E0DF91CF911F91C2CEDF91CF91E7
:100550001F910895EF92FF920F931F93CF938630D0
:1005600018F006E910E002C00AEF10E07801EE0C86
:10057000FF1CC82FCC23D1F019BC18BC1BBCC80170
:10058000A7DE8091CD00882321F08091E5000EDF69
:1005900009C08091FD009091CA002091E40029BD1E
:1005A00098BD8BBDC70194DEC150E4CFCF911F91A0
:1005B0000F91FF90EF900895CF93C82F68E270E0FD
:1005C00082E053DF80EF90E083DE64E670E08C2F02
:1005D0004CDF1092BC00CF91089586B383FB88272F
:1005E00080F991E098278091A400880F892B80934F
:1005F000A4009091A300992311F08F7001C0817025
:100600008093A3008091A30090E008958091BB00A7
:10061000803120F48091BB008093BA008091BB00B0
:100620008F5F8093BB009091E200891710F01092C9
:10063000BB0008958091BB008093BA008091BB00FD
:10064000811103C08091E20002C08091BB00815003
:100650008093BB00089518958EBB6DBB84E28CBB64
:1006600086E28CBBE199FECF0895CF93DF93209172
:10067000BB008091F7009091CD00880F880F880F04
:10068000979599279795692F682B622B6093F800AF
:100690002091CC003091FA009091FB008091CB002A
:1006A000330F990F990F932B922B8295880F807E91
:1006B000892B8093C9004091C8005091F600309179
:1006C000F9009091E3008091FC007091E600550FD5
:1006D000330F330F352B342B990F990F990F292F87
:1006E000232B8295807F982F922B872F8295880FBE
:1006F000807E892B8093F400C091A500D091A60044
:10070000CE0104968F7799279093A6008093A50039
:10071000A3DF8091A5006091C9008F5F9DDF80916C
:10072000A5006091F4008E5F97DFCEBB84E18CBBA7
:1007300086E18CBBE199FECF8C2F8F5F8EBB84E16D
:100740008CBB86E18CBBE199FECF8C2F8E5F8EBB7C
:1007500084E18CBB86E18CBBE199FECFCD5FCEBB43
:1007600084E18CBB86E18CBBE199FECF8091A50032
:100770006DE58D5FDF91CF916FCF1F920F920FB616
:100780000F9211242F933F938F939F9384B195B130
:100790002091AA00213039F49C0136952795369591
:1007A00027952093AC002091AA002330E1F48E51CC
:1007B00091402091AB002223A1F02091AB0030E0CA
:1007C0002817390728F42091AB002F5F2093AB0046
:1007D0002091AB0030E08217930728F48091AB00A2
:1007E00081508093AB008091AA008F5F8093AA0014
:1007F000843010F01092AA008091AA00823010F488
:1008000081E801C08FE887B99F918F913F912F9127
:100810000F900FBE0F901F9018951F920F920FB65A
:100820000F9211242F933F934F935F936F937F9376
:100830008F939F93AF93BF93EF93FF938091F500B6
:10084000882321F081508093F500B5C48091A800E1
:100850009091A900892B49F08091A8009091A9005E
:1008600001979093A9008093A800B7DE2091B7006C
:100870003091B800892B09F4E1C1203D87E03807A9
:1008800030F42F5F3F4F3093B8002093B700809132
:10089000B7009091B800823E24E0920791F4209135
:1008A000C70021110EC01092C6001092E5001092F0
:1008B000BB001092C50081E08093C0001092BF0081
:1008C0007AC43091BF002091B0003323B1F0109270
:1008D000BC00211170C48332910521F48091BF00C6
:1008E0008F5F08C08634910509F065C481E080936C
:1008F000B0008FE08093BF005EC4211194C12091AD
:10090000C700222349F0019709F0A3C08091C000DD
:1009100081119FC086E974C02091CD00222309F483
:1009200098C0429708F495C08091C000811191C091
:100930008091C10081118DC08091BB00803508F08D
:1009400088C01092A2008091C500813009F44DC08A
:1009500038F0823009F457C0833009F45EC079C0A2
:100960008091C60081111BC081E08093C50087E1A2
:100970008093E7008091FB0089BD18BC1BBC8FEF02
:100980008093C6008093E5008091C200811104C06D
:100990008091C6008093C2001092C3005AC080911B
:1009A000C3009091C400882329F09093C500109251
:1009B000C30004C085E0891B8093C5008091C600F8
:1009C0008F3FD1F08091C600863938F083E0809364
:1009D000C50086E98093E5003BC08091C600813068
:1009E000C1F582E08093C50034C08091E70081505A
:1009F0008093E70081112DC082E08093C50081E0E3
:100A00008093C600E7CF8093C4008091C6008639EA
:100A1000B0F48091C6008F5F09C08093C4008091BC
:100A2000C600823060F08091C60081508093C6007D
:100A30008093E5008091C6008093C20007C084E0E7
:100A40008093C50041DC87E090E042DC8091E500C6
:100A5000ADDC8091CD00811135C08091B7009091BF
:100A6000B800489779F58091C00081112BC0809122
:100A7000BB00803190F48091C70081110EC080913D
:100A8000CC00882311F0C2DD1DC08091BB008130F5
:100A900011F41092BB00CEDD15C08091BB008B35E8
:100AA00088F08091FE00811102C080916300815026
:100AB0008093FE00E091FE00F0E0EC56FF4F808155
:100AC0008093BB008091B7009091B8008B34910562
:100AD00009F075C08091B600823009F58091B300AD
:100AE0009091B4000E97D8F48091CD00882329F01E
:100AF0008091C000813009F062C01092C60010924F
:100B0000E5001092BB001092C5009091C00081E0FA
:100B1000282F291B2093C0008093C10050C08091D2
:100B2000C00081114CC08091B6008130A1F42091A9
:100B3000B3003091B4002E30310568F49091CD00AF
:100B400091113DC090E59093BB008093C10019BC0A
:100B500018BC1BBC34C08091BB008B3510F073DC1B
:100B60002EC08091BB00803539F41092BB0019BCB7
:100B700018BC1BBC85E10AC08091BB00823571F4B2
:100B80001092BB0019BC18BC1BBC8EE08093BF0048
:100B90001092BD0081E08093B00011C08091CD0023
:100BA00081110DC08091E600882349F08091BB003F
:100BB000803529F08091C700811101C038DC809117
:100BC000C000811130C08091C70081112CC080917C
:100BD000CD0081110FC08091B7009091B800883C82
:100BE000910541F48091B600823021F08091BB00E4
:100BF000803559F48091CD008823A9F08091B70009
:100C00009091B800843F914071F41092BB00109213
:100C1000C6001092C50019BC18BC1BBC81E08093B3
:100C2000BF001092BD001092A1001092A00088E3B6
:100C300091E09093610080936000B3C21092B00085
:100C40008091BF008823A1F02115310559F028318A
:100C5000310528F48091BD008F5F8093BD00109214
:100C6000BC009BC28091BC008F5F8093BC0095C28A
:100C7000232B09F41BC18091C700882329F010920F
:100C8000C6001092E50020DB2091CD008091B700D6
:100C90009091B800222309F476C01092C5004297C3
:100CA00008F06CC08091B6008F5F8093B600809191
:100CB000B600813009F064C08091BB0080939F0032
:100CC0008091BB00803138F48091C600863919F4D8
:100CD0008FEF80939F008091BB00803541F0809121
:100CE000BB00813521F08091BB00823549F4109220
:100CF000BB001092C6001092E50081E08093C10015
:100D00008091C60080939E008091C000811138C000
:100D10008091C100811134C08091C700811130C021
:100D20008091C60081111AC08091C200811103C058
:100D300081E08093C20081E08093C30082E08093D1
:100D4000C4008091C2008093C6008093E50089EAC8
:100D500093E09093A9008093A80004C01092C6006D
:100D60001092E5008091E5008F3F31F48091FB0007
:100D700089BD18BC1BBC04C019DB02C01092B600B0
:100D80001092C1008EC0489708F089C08091BB00C6
:100D9000803541F08091BB00813521F08091BB000E
:100DA000823561F48091BB0080939F001092BB005C
:100DB0008091B6008F5F8093B60073C08091BB00B6
:100DC000811106C08091B600811102C081E007C088
:100DD0008091B600882329F08091B6008F5F8093C0
:100DE000B6008091C00081115CC08091FA00882318
:100DF00099F08091B500882379F08091BB00811132
:100E00000BC08091C70081114CC08091B5008093C8
:100E1000BB001092B50045C08091BB00803110F539
:100E20008091C70081113DC08091BB00882391F063
:100E30008091B3009091B4008B34910558F080916B
:100E4000BB008093B5008091BB008093BA001092E4
:100E5000BB0027C08091CC00882311F0EBDB21C0C0
:100E6000D5DB1FC08091B3009091B4008B34910505
:100E700010F0E9DA16C08091E6008130D1F3E091FC
:100E8000FE00EF5FE093FE0080916300E81788F7B3
:100E9000F0E0EC56FF4F80818093BB0002C01092BF
:100EA000B6001092B4001092B30077C18091B300E5
:100EB0009091B40001969093B4008093B300892B75
:100EC00031F480E395E79093B4008093B300809170
:100ED000B3009091B4000F9708F4A6C08091B600BB
:100EE0008530B9F48091CD00882309F49BC08091AE
:100EF000C000811197C08091C700811193C081E02B
:100F00008093C7001092C6001092E5001092BB00BB
:100F100038C08091B6008430F9F48091CD00811101
:100F200005C08091C000882309F47CC08091C7006F
:100F3000811178C01092C6001092E5001092BB009B
:100F40001092C5009091C00081E0282F291B2093AA
:100F5000C0008093C10066C080919F0090EB980F05
:100F6000923098F49091B600923009F05BC08035D1
:100F700011F481E501C082E58093BB0081E080939C
:100F8000C10019BC18BC1BBC4DC08091CD0088238A
:100F900009F448C08091C000811144C08091C7000D
:100FA000811140C08091B600833049F480E5809380
:100FB000BB0081E08093C10019BC18BC1BBC8091B0
:100FC000B600823079F580919F008F3FC9F48091FF
:100FD000E600882311F02BDA25C08091C200863903
:100FE00039F08091A2008093C6008093E50004C090
:100FF0001092C6001092E5008091E500D7D912C08A
:1010000086E98093C6008091C6008093E500CED922
:1010100080919E008093A20089EA93E09093A900BA
:101020008093A8001092B6008091CB008230E8F146
:101030008091CD008823E1F08091E50088588737C2
:10104000A0F58091A0009091A10001969093A1003D
:101050008093A0002091B1003091B2002817390789
:1010600020F58EE78093C6008093E5009FD91DC0D0
:101070008091BB008031C8F4E091BB00F0E0E25306
:10108000FF4F80818F3F89F48091A0009091A10053
:1010900001969093A1008093A0002091B10030911F
:1010A000B2002817390708F4C5DA8091CD008823EB
:1010B00091F08091C600823070F08091C600863930
:1010C00050F48091B3009091B4008C34910518F0E5
:1010D00081E08093C300809160009091610000974F
:1010E00029F00197909361008093600080916000E7
:1010F00090916100892BD1F59091BB008091CD003A
:10110000811104C081E0913041F408C09091E50064
:1011100081E0913019F09F3F09F080E02091AC0010
:1011200030E0811103C08BEA90E002C081EA90E0D8
:101130002817390734F480919D008F5F80939D00BC
:1011400004C010929D001092AE0080919D008830E6
:1011500068F081E08093AF008093AE0010929D0014
:1011600088E391E090936100809360008091AE00ED
:10117000882399F080919B0090919C000196909318
:101180009C0080939B00843F914039F481E08093E0
:10119000AD0010929C0010929B001092B80010922B
:1011A000B70080919A008F5F80939A00837019F442
:1011B00086B1886486B9FF91EF91BF91AF919F91FD
:1011C0008F917F916F915F914F913F912F910F90F0
:1011D0000FBE0F901F90189517BA88E088BB85BB8B
:1011E00083E187BB81EA8ABD81E083BF80BF80E65F
:1011F0008CBD8FEF8DBD81E887B9A29A87EC86B947
:10120000479A85B7877E806185BFF8948BB78F7DBD
:101210008BBFA89584B7877F84BF81B5886181BD66
:1012200011BCD9D81092A6001092A5000091A5007B
:101230001091A6000038110508F0DDC4C80113D5CF
:10124000F82E8093F800C80101960DD5D82F809311
:10125000C900C801029607D5C82F8093F400C801C1
:10126000039601D58D3539F00C5F1F4F1093A60002
:101270000093A500DBCF8F2D87708093BB008F2D4F
:101280008695869586958F708093F700FF1CFF24C6
:10129000FF1CF092CD008D2F81708093CC00D1FB8C
:1012A000882780F98093FA008D2F86958695877020
:1012B0008093FB00D295D695D770D093CB008C2F1E
:1012C00081708093C800C1FB882780F98093F60065
:1012D000C2FB882780F98093F900C3FB882780F937
:1012E0008093E300C4FB882780F98093FC00C295BB
:1012F000C695C370C093E6008091F9008093F20018
:101300008AEF90E0B0D49FEF980F9E3F10F4809347
:101310006200E7D7E091CB00F0E0EE0FFF1FE45A48
:10132000FF4F859194919093B2008093B10080918A
:10133000C800882359F08091CD00811107C08091A9
:10134000FF00811105C062D990D902C01092BB0084
:101350008091BB0081110CC08091CD00811104C02F
:101360008091C800811104C060E570E082E07DD802
:101370001092FF008AEF8093F30089E18093F500DB
:10138000F894A89581B5886181BD80E481BD789489
:10139000812C912C00E0C1E0DFE0B8E25B2E1FEF72
:1013A00088E3C82EDD24D3949CEFE92E9AE0F92E31
:1013B00025E0A22EB12C44244A948091BF008111D3
:1013C00040C28091C0000817B1F00091C00019BC64
:1013D00018BC1BBC6BE470E084E047D81092C100DD
:1013E0008091C000882329F08091BB008093F30096
:1013F00002C04092F3008091C700981669F0909067
:10140000C7006CE370E082E030D88AEF90E060D7EC
:101410006BE470E083E029D89091BB008091F300E9
:10142000981709F414C18091BB00803118F58091A0
:10143000BB0090E0FC01E852FF4F20812093E400C4
:10144000FC01E851FF4F20812093CA00FC01E253C8
:10145000FF4F80818093FD008091FD009091CA0034
:101460002091E40029BD98BD8BBD8091BB00809385
:10147000F300EDC08091BB008093F30019BC18BC51
:101480001BBC8091BB00803501F580E991E020D73D
:101490001092C1008091BB00803509F0D8C080E077
:1014A0009091AC00E82FF0E0E45DFF4FE491E91784
:1014B00010F48E5FF5CF81118250E82FF0E0E35DEC
:1014C000FF4F849160E525D8E5CF8091BB00813541
:1014D00079F48AEF90E0FCD61092C1008091BB00B5
:1014E000813509F0B4C08091AB0061E512D8F6CF28
:1014F0008091BB00823571F48AEF90E0E9D61092BA
:10150000C1008091BB00823509F0A1C062E58CE08A
:1015100000D8F7CF8091BB008B3549F48091BB0098
:101520008B3509F094C069E28EE06FD7F7CF8091D8
:10153000BB008C3501F58091BB008C3509F087C06C
:10154000A8E07A2E8091BB008C3519F0F8E07F2E50
:101550000DC068E284E159D77A947110F3CFF6CFC9
:1015600060E588E252D77A94772029F38091BB0016
:101570008C35B1F3E0CF8091BB008D3561F5809162
:10158000BB008D3521F5E4E07E2E8091BB008D35CA
:1015900019F07AE0772E16C019BC18BC1BBD85E087
:1015A00090E096D619BD18BC1BBC81E490E090D6A3
:1015B0007A947110EACFEDCF88E490E089D67A94DE
:1015C0007720E9F28091BB008D35B1F3D8CF19BCFB
:1015D00018BC1BBC3CC08091BB008E35D1F48091FF
:1015E000BB008E35A1F58CE291E072D66DE78DE7F8
:1015F0000CD76DE78DE709D76FE0762E8091BB00A1
:101600008E3569F784E690E063D67A947110F6CF50
:10161000E6CF8091BB008F35D1F48091BB008F3530
:10162000B1F48CE291E054D660EF80EFEED660EF3B
:1016300080EFEBD654E6752E8091BB008F3569F7AD
:1016400084E690E045D67A947110F6CFE6CF80918B
:10165000AF00882309F445C08091CD00882369F14B
:101660008091E5008823D1F1813011F08F3F61F442
:1016700087E08093E50088E06DD71092C600109255
:10168000E5001092C50012C083E064D78091E500A8
:101690008A3050F090E0880F991F880F991FB5018C
:1016A000BBD26093E50002C0C093E5008091E500E5
:1016B0007DD68AEF90E00CD611C08091BB008823C4
:1016C00069F08091BB00813011F488E001C083E0B3
:1016D00041D78091BB00803108F4ACD71092AF00A5
:1016E00005C08091AD0081111092AD008091CB00BA
:1016F0008130A9F59091AB0080916200981778F144
:101700008091A8009091A900892B49F58091CD0086
:101710008823C1F08091E5009FE8980F9E38F8F487
:10172000282F30E066E06CD2A901481B5109CA019C
:10173000413751050CF480E78093E5008091E50086
:1017400035D609C08091BB00882349F08091BB0049
:10175000803128F46FD7F092A900E092A800809120
:10176000AE00882329F034EE632E37E5732E04C0D3
:1017700026E3622E772473948091CD00811104C0FA
:101780008091BB00882349F08091CD00882309F423
:1017900050C08091E50081114CC01FD7892B09F002
:1017A00048C08091B3009091B4006816790608F0A3
:1017B00040C081E090E08CD51092B4001092B3004C
:1017C0001092A9001092A800F894A89584B7877F7A
:1017D00084BF81B5886181BD11BC7894379810921F
:1017E000B8001092B700F9D6892B21F080E190E083
:1017F0006FD5F9CF8BB780628BBF85B7806285BF0D
:1018000085B7846885BF8B7F85BF889585B78F7DB9
:1018100085BF8BB78F7D8BBF81E887B9A29A87EC94
:1018200086B9F894A89581B5886181BD80E481BDB1
:1018300078948091A700882309F4BFCD1092A70067
:10184000BCCD8091BD00881581F08090BD00809155
:10185000BD00882351F084E189BD18BC1BBC84E61F
:1018600090E036D519BC18BC1BBC9091BF0080918C
:10187000BE00981709F4A3C18091BF008093BE00F9
:101880001092BC008091BF00873109F47CC0E0F465
:101890008E3009F448C028F4813059F1833091F139
:1018A000E1C08F3009F45AC0853109F0DBC080E90E
:1018B00091E00ED581E080D68091BF008F5F80934C
:1018C000BF001092BD0078C1883209F475C138F4A8
:1018D000883109F467C0893109F471C0C3C0843606
:1018E00009F479C0853609F482C0893209F0BAC09A
:1018F0008EC080E991E0ECD481E05ED68091BF009B
:101900008F5F3CC18091BD00882359F08091BD005C
:10191000893038F48091BD0081708C278093CD0090
:10192000A4D682E039C157D5A0D68091F900809322
:10193000F200D7D48CE3809362006CE38AEF8CD6FC
:10194000E091CB00F0E0EE0FFF1FE45AFF4F8591CE
:1019500094919093B2008093B1002CC11092BF007B
:1019600068E270E085E081D51092C6001092E50033
:101970001092BB008091CD00882309F41DC1809195
:10198000C60014D519C18091BD00882351F2809101
:10199000BD0081708C278093F9008091F9008093BD
:1019A000F200BECF8091BD00882339F08091BD0048
:1019B00081708C278093E30058D683E0EDC080913E
:1019C000BD00882309F4F6C08091BD0081708C278A
:1019D0008093F600EEC068E270E083E046D519BC63
:1019E00018BC1BBDD092A900C092A800E5C019BCCC
:1019F00018BC1BBC8091A8009091A900892B11F5FF
:101A00006091AB00609362008AEF26D61BC0809184
:101A1000BD008823B9F08091BD00873098F4809193
:101A2000BD008F5F8093CB0020D6E091CB00F0E02B
:101A3000EE0FFF1FE45AFF4F859194919093B200EF
:101A40008093B1008091CD00882321F084E0B4D54B
:101A500085E003C088E0B0D589E08093BF00809323
:101A6000BE00AAC08091CD008823C1F18091BF0043
:101A70008530A1F0863079F1843009F09DC08091E5
:101A8000BD00882309F499CF8091BD00883008F00B
:101A900094CF8091BD008093FB003CC08091BD003D
:101AA000813019F41092CB0013C08091BD008230B8
:101AB00009F460C08091BD00833059F466C088236A
:101AC00041F08091BD0081708C278093FC0009D487
:101AD000CCD584E061C08091BD0060C0E091BF00C2
:101AE0008E2F90E0FC013497E730F10508F064C0D8
:101AF000E15FFF4F8091BD000994882309F45DCF19
:101B00008091BD008D3008F058CF8091BD0081508C
:101B10008093F700E6D350CF882339F08091BD0041
:101B200081708C278093CC00A0D585E035C08823B8
:101B300039F08091BD0081708C278093FA0095D593
:101B400086E02AC0882351F08091BD00883030F4AF
:101B50008091BD008093FB00C4D387D587E01CC073
:101B6000813021F41092CB0080D515C08091BD004A
:101B7000823039F4C093CB0078D584E68093BF00DF
:101B80001BC08091BD00833031F468E270E06DD4F9
:101B90005092BF0011C088E00FD50EC0882351F0CD
:101BA0008091BD00843030F48091BD0081508093DD
:101BB000E6005BD5D093BF001092BD00FECB8091B4
:101BC000BD00882321F08091BC008E3770F4809195
:101BD000BF00843609F4F1CB8091BD008111EDCBBB
:101BE0008091BC008C3D08F4E8CB8091BF008F5FF2
:101BF0008093BF00E2CB1092A6001092A5007CCB90
:101C0000991B79E004C0991F961708F0961B881F4E
:101C10007A95C9F78095089597FB072E16F40094DE
:101C200006D077FD08D00BD007FC05D03EF4909588
:101C300081959F4F0895709561957F4F0895AA1BD8
:101C4000BB1B51E107C0AA1FBB1FA617B70710F0A7
:101C5000A61BB70B881F991F5A95A9F780959095D9
:101C6000BC01CD010895E199FECF9FBB8EBBE09AE8
:0A1C700099278DB30895F894FFCF73
:101C7A0038013C05CB00C500BC00B000A1008F00B4
:101C8A007A007400CC00C700BF00B400A60095001B
:101C9A0081007600CD00C900C200B800AB009B00ED
:0A1CAA00880078005B5C5D5E5F005F
:00000001FF
